:0200000480007A
:100000006F008004732F2034930F80006308FF0378
:10001000930F90006304FF03930FB0006300FF038E
:10002000130F000063040F0067000F00732F2034CC
:1000300063540F006F00400093E19153171F0000BD
:1000400023223FFC6FF09FFF93000000130100008C
:10005000930100001302000093020000130300004C
:100060009303000013040000930400001305000034
:10007000930500001306000093060000130700001C
:100080009307000013080000930800001309000004
:1000900093090000130A0000930A0000130B0000EC
:1000A000930B0000130C0000930C0000130D0000D4
:1000B000930D0000130E0000930E0000130F0000BC
:1000C000930F0000732540F16310050097020000B4
:1000D000938202017390523073500018970200000F
:1000E0009382020273905230B70200809382F2FF33
:1000F0007390023B9302F0017390023A73504030C8
:100100009702000093824201739052307350203066
:100110007350303093010000970200009382C2EECA
:1001200073905230130510001315F501634C050050
:100130000F00F00F930110009308D0051305000085
:100140007300000093020000638A02007390521053
:10015000B7B2000093829210739022307350003037
:10016000970200009382420173901234732540F18C
:1001700073002030930000001301000033A720001B
:100180009303000093012000631A774A9300100044
:100190001301100033A720009303000093013000E7
:1001A000631E7748930030001301700033A72000CE
:1001B000930310009301400063127748930070008E
:1001C0001301300033A72000930300009301500077
:1001D00063167746930000003781FFFF33A72000A6
:1001E0009303000093016000631A7744B700008016
:1001F0001301000033A72000930310009301700047
:10020000631E7742B70000803781FFFF33A72000CD
:100210009303100093018000631277429300000063
:10022000378100001301F1FF33A720009303100072
:100230009301900063147740B70000809380F0FF33
:100240001301000033A72000930300009301A000D6
:100250006316773EB70000809380F0FF378100007F
:100260001301F1FF33A72000930300009301B000B6
:100270006316773CB7000080378100001301F1FF5F
:1002800033A72000930310009301C0006318773A4E
:10029000B70000809380F0FF3781FFFF33A7200075
:1002A000930300009301D000631A77389300000095
:1002B0001301F0FF33A72000930300009301E00037
:1002C000631E77369300F0FF1301100033A7200060
:1002D000930310009301F000631277369300F0FF50
:1002E0001301F0FF33A720009303000093010001E6
:1002F000631677349300E0001301D000B3A0200010
:100300009303000093011001639A70329300B000D0
:100310001301D00033A120009303100093012001AA
:10032000631E71309300D000B3A01000930300004F
:100330009301300163947030130200009300B00009
:100340001301D00033A7200013030700130212008B
:1003500093022000E31452FE930310009301400126
:10036000631E732C130200009300E0001301D00001
:1003700033A720001300000013030700130212002C
:1003800093022000E31252FE9303000093015001F8
:100390006316732A130200009300C0001301D000FB
:1003A00033A7200013000000130000001303070010
:1003B0001302120093022000E31052FE9303100078
:1003C00093016001631C7326130200009300E00098
:1003D0001301D00033A72000130212009302200063
:1003E000E31652FE93030000930170016318772413
:1003F000130200009300B0001301D00013000000AE
:1004000033A720001302120093022000E31452FECF
:1004100093031000930180016312772213020000FE
:100420009300F0001301D00013000000130000003F
:1004300033A720001302120093022000E31252FEA1
:100440009303000093019001631A771E13020000CA
:100450009300A000130000001301D00033A7200078
:100460001302120093022000E31452FE93031000C3
:100470009301A0016314771C130200009300000194
:10048000130000001301D0001300000033A7200068
:100490001302120093022000E31252FE93030000A5
:1004A0009301B001631C77181302000093009000C1
:1004B00013000000130000001301D00033A7200038
:1004C0001302120093022000E31252FE9303100065
:1004D0009301C00163147716130200001301D000CA
:1004E0009300100133A72000130212009302200092
:1004F000E31652FE930300009301D00163107714BA
:10050000130200001301D0009300800013000000CC
:1005100033A720001302120093022000E31452FEBE
:10052000930310009301E001631A77101302000097
:100530001301D000930020011300000013000000FD
:1005400033A720001302120093022000E31252FE90
:10055000930300009301F0016312770E1302000071
:100560001301D000130000009300700033A7200097
:100570001302120093022000E31452FE93031000B2
:1005800093010002631C770A130200001301D000DC
:1005900013000000930030011300000033A7200077
:1005A0001302120093022000E31252FE9303000094
:1005B0009301100263147708130200001301D000A6
:1005C00013000000130000009300600033A7200018
:1005D0001302120093022000E31252FE9303100054
:1005E00093012002631C77049300F0FF3321100075
:1005F0009303000093013002631271049300F0FF33
:1006000033A10000930310009301400263187102AC
:10061000B320000093030000930150026390700226
:10062000930000011301E00133A0200093030000B8
:100630009301600263147000631030020F00F00F2A
:10064000638001009391110093E111009308D0059C
:1006500013850100730000000F00F00F93011000DC
:100660009308D0051305000073000000731000C04C
:0C0670000000000000000000000000007E
:1010000000000000000000000000000000000000E0
:1010100000000000000000000000000000000000D0
:1010200000000000000000000000000000000000C0
:1010300000000000000000000000000000000000B0
:081040000000000000000000A8
:040000058000000077
:00000001FF
